:03000000022000DB
:10070000C2C07800790020B008D8FBD9F9758902F9
:060710002243B10280FE4D
:0F076000C2B43099FBC299F5993099FDD2B422F9
:1020000075890275C830E4F5CDF5CC30B0FD20B04F
:10201000FDD2CA30B0FDC2CAE5CCC4540FF8E5CD3C
:10202000C454F048F4F5CCF5CAE5CDC4540FF4F52A
:10203000CDF5CBD2CA7598523098FDC298E5995427
:102040007F122117B455F190212912211F758E009E
:1020500053B1FC900003E493FF900044E493FE909E
:10206000213EBFC209900047E493FE90214E122109
:102070001FBE120890216A12211F80FE900000E40A
:1020800093F0A3E58270F843B101BFC21E900047F0
:102090007412F0A37407F0A37400F09000D57402DA
:1020A000F0A37407F0A37460F0801C9000447412D5
:1020B000F0A37407F0A37400F09000D27402F0A3B0
:1020C0007407F0A37460F090000011F59000801187
:1020D000F590070011F5900000E03103A3E5827050
:1020E000F8900700E4933103A3E582B480F69021D1
:1020F0005E311F80FE43B1408583B48582B375B2E3
:102100000B800E43B1408583B48582B3F5B575B2BB
:102110000EE5B620E2FB223099FDC299F59922E442
:102120009360053117A380F7220D0A53746172740E
:10213000207061746368696E672E2E2E20005634FD
:102140002064657465637465642E2E2E20005635F8
:102150002064657465637465642E2E2E20005061C2
:1021600074636820646F6E652E00416C72656164F3
:10217000792070617463686564202D206E6F206122
:072180006374696F6E2E000D
:00000001FF
